:1000000029C043C042C041C040C03FC03EC03DC007
:100010003CC03BC03AC039C038C037C036C035C01C
:1000200034C033C032C0084AD73B3BCE016E84BCDB
:10003000BFFDC12F3D6C74319ABD56833DDA3D0042
:10004000C77F11BED9E4BB4C3E916BAAAABE00008B
:1000500000803F0011241FBECFE5D4E0DEBFCDBF3E
:1000600011E0A8E6B1E001C01D92AC3AB107E1F79A
:1000700011E0A0E6B0E0ECEFFDE102C005900D92CA
:10008000A836B107D9F701D2B7CEBACFA59A8AE080
:10009000982F9A95F1F7A49A982F9A95F1F7A59829
:1000A000982F9A95F1F7A4988A95F1F71092680124
:1000B0009C9905C0809168018F5F809368019D992C
:1000C00005C0809168018F5F809368018AE0982F56
:1000D0009A95F1F7982F9A95F1F7982F9A95F1F74D
:1000E0008A95F1F70895A498A598AC98AD98CEDFBD
:1000F000CDDF0895A49A8AE0982F9A95F1F7A59AF2
:100100008A95F1F70895A4988AE0982F9A95F1F7C7
:10011000A598982F9A95F1F7A49A982F9A95F1F7A8
:10012000A59A8A95F1F7089520E04AE087FD02C07C
:10013000A49A01C0A4983AE0942F9A95F1F7A59853
:10014000942F9A95F1F7A59A2F5F283011F0880F18
:10015000EDCFA498832F8A95F1F7A598832F8A95E0
:10016000F1F783B3A59A90E024E0969587952A95B8
:10017000E1F781700895A49820E030E04AE0330F61
:10018000A598942F9A95F1F79C993160A59A942F90
:100190009A95F1F72F5F283091F7882311F4A49AEC
:1001A00001C0A4988AE0982F9A95F1F7A598982F06
:1001B0009A95F1F7A59A8A95F1F7A498832F089557
:1001C0000F931F93182F062F95DF80EDADDF812F42
:1001D000ABDF802FA9DF5ADF1F910F91089589E1CE
:1001E00067E0EEDF8AE160E0EBDF8BE168E1E8DF0A
:1001F0008CE160E0E5DF8DE160E0E2DF8EE160E070
:10020000DFDF8FE160E0DCDF80E260E0D9DF81E208
:1002100060E0D6DF82E260E0D3DF83E260E0D0DF3F
:1002200084E260E0CDDF85E260E0CADF86E260E084
:10023000C7DF87E260E0C4DF88E260E0C1DF89E217
:1002400060E0BEDF8AE260E0BBDF8BE260E0B8DF47
:100250008CE260E0B5DF8DE260E0B2DF8EE260E06C
:10026000AFDF8FE260E0ACDF80E360E0A9DF81E335
:1002700060E0A6DF82E360E0A3DF83E360E0A0DF6D
:1002800084E360E09DDF85E360E09ADF87E360E080
:1002900097DF88E360E094DF83E660E091DF84E647
:1002A00060E08EDF85E660E08BDF86E660E088DF79
:1002B00087E660E085DF88E660E082DF89E660E06F
:1002C0007FDF8AE660E07CDF8BE662E079DF8CE648
:1002D00060E076DF08950EDF80ED26DF8BE324DF1C
:1002E000D5DE08DF81ED20DF80E045DF8093A001CF
:1002F00080E041DF8093870180E03DDF80937901DA
:1003000080E039DF80939F0180E035DF80938901B1
:1003100081E031DF8093A101B9DE9091A00180E0FE
:1003200020918701820F911DAA2797FDA095BA2FD2
:1003300080939A0190939B01A0939C01B0939D019F
:100340009091790180E020919F01820F911DAA2751
:1003500097FDA095BA2F8093810190938201A0937D
:100360008301B09384019091890180E02091A101E3
:10037000820F911DAA2797FDA095BA2F80938E0119
:1003800090938F01A0939001B09391010895B2DEF4
:1003900080EDCADE83E4C8DE79DEACDE81EDC4DE4A
:1003A00080E0E9DE8093A30180E0E5DE8093A20196
:1003B00080E0E1DE8093880180E0DDDE80938001D3
:1003C00080E0D9DE8093860181E0D5DE80937A01DA
:1003D0005DDE9091A30180E02091A201820F911D2A
:1003E000AA2797FDA095BA2F809396019093970125
:1003F000A0939801B09399019091880180E0209199
:100400008001820F911DAA2797FDA095BA2F809396
:10041000A4019093A501A093A601B093A701909188
:10042000860180E020917A01820F911DAA2797FD15
:10043000A095BA2F80937B0190937C01A0937D01BE
:10044000B0937E01089556DE80ED6EDE81E46CDEB1
:100450001DDE50DE81ED68DE80E08DDE80939E0142
:1004600081E089DE8093850111DE089543DE80ED11
:100470005BDE85E759DE0ADE3DDE81ED55DE81E09B
:100480007ADE80937F0102DE08952F923F924F9291
:100490005F926F927F928F929F92AF92BF92CF9214
:1004A000DF92EF92FF920F931F93DF93CF93CDB71D
:1004B000DEB728970FB6F894DEBF0FBECDBF8FE32F
:1004C00087BB18BA5BD40FDE8ADE81E04BD480EAAA
:1004D0009FE00197F1F7B7DF60918501772767FD0E
:1004E0007095872F972F64587F4C8F4F9F4F209187
:1004F0009E01332727FD3095322F2227442737FDD1
:100500004095542F620F731F841F951F24E531E01F
:1005100040E050E03DDA209375013093760140933E
:1005200077015093780184E91DD484E721D48DE3C9
:100530001FD480917501D9D3CEDE20909A013090DE
:100540009B0140909C0150909D0180918101909170
:100550008201A0918301B09184018D839E83AF833A
:10056000B887BC01CD01ADD79B01AC010ED67B0194
:100570008C0160908E0170908F018090900190901E
:100580009101C401B3019DD79B01AC01FED55B0174
:100590006C01C801B701A6019501D0D537DB7B01FD
:1005A0008C0166277727CB016219730984099509A5
:1005B00088D7A8019701DED65FDA24E13EE245E65E
:1005C00052E4E3D5D8D769837A838B839C83609385
:1005D000A8017093A9018093AA019093AB01C20175
:1005E000B1016FD79B01AC01D0D59B01AC01CA0111
:1005F000A6019501A3D50ADB7B018C016D817E816B
:100600008F81988590958095709561957F4F8F4FDC
:100610009F4F57D7A8019701ADD62EDA24E13EE2CD
:1006200045E652E4B2D5A7D760938A0170938B0157
:1006300080938C0190938D01C201B10142D79B013F
:10064000AC01A3D57B018C016D817E818F81988562
:1006500038D79B01AC0199D59B01AC01C801B7010A
:100660006DD5D4DA7B018C01909480947094609461
:10067000611C711C811C911CC401B30122D7A8010B
:10068000970178D6F9D924E13EE245E652E47DD5DA
:1006900072D7609392017093930180939401909329
:1006A000950189819A81AB81BC81865A9F4FAF4F5A
:1006B000BF4F4E97A105B10510F4C09AC19889812A
:1006C0009A81AB81BC81CC96A11DB11D4E97A1052D
:1006D000B10510F4C19AC29889819A81AB81BC811D
:1006E0004E96A11DB11D4E97A105B10510F4C29AF9
:1006F000C39889819A81AB81BC814E97A105B105D0
:1007000010F4C39AC49889819A81AB81BC814E97B9
:10071000A109B1094E97A105B10510F4C49AC59875
:1007200089819A81AB81BC81CC97A109B1094E978F
:10073000A105B10508F4C59A80E814D381E418D363
:1007400080919A0190919B01A0919C01B0919D0193
:10075000B7FF1CC082E806D38DE20AD380919A01CC
:1007600090919B01A0919C01B0919D01B095A095A5
:10077000909581959F4FAF4FBF4F80939A01909373
:100780009B01A0939C01B0939D0104C082E8EAD232
:100790008BE2EED28091810190918201A091830140
:1007A000B0918401B7FF1CC088E8DCD28DE2E0D2B2
:1007B0008091810190918201A0918301B091840187
:1007C000B095A095909581959F4FAF4FBF4F809367
:1007D000810190938201A0938301B093840104C0AE
:1007E00088E8C0D28BE2C4D280918E0190918F01B3
:1007F000A0919001B0919101B7FF1CC08EE8B2D2D8
:100800008DE2B6D280918E0190918F01A0919001DE
:10081000B0919101B095A095909581959F4FAF4F64
:10082000BF4F80938E0190938F01A0939001B0935E
:10083000910104C08EE896D28BE29AD283E892D2DC
:1008400060919A0170919B0180919C0190919D0112
:1008500028E030E040E050E09BD8DA01C901B6D191
:100860008AE386D289E87ED260918101709182010B
:10087000809183019091840128E030E040E050E0D5
:1008800087D8DA01C901A2D18AE372D28FE86AD28D
:1008900060918E0170918F018091900190919101F2
:1008A00028E030E040E050E073D8DA01C9018ED191
:1008B0006EDD60917B0170917C0180917D01909152
:1008C0007E0126E130E040E050E062D88091710185
:1008D00090917201A0917301B0917401820F931FE6
:1008E000A41FB51F8093710190937201A0937301AF
:1008F000B093740183EE36D26091710170917201F0
:1009000080917301909174012AE030E040E050E062
:100910003FD8DA01C9015AD180EC24D287E428D229
:100920008091960190919701A0919801B0919901C1
:10093000B7FF1CC082EC16D28DE21AD280919601CC
:1009400090919701A0919801B0919901B095A095CF
:10095000909581959F4FAF4FBF4F80939601909395
:100960009701A0939801B093990104C082ECFAD149
:100970008BE2FED18091A4019091A501A091A601E6
:10098000B091A701B7FF1CC088ECECD18DE2F0D18B
:100990008091A4019091A501A091A601B091A70119
:1009A000B095A095909581959F4FAF4FBF4F809385
:1009B000A4019093A501A093A601B093A70104C040
:1009C00088ECD0D18BE2D4D180917B0190917C01D5
:1009D000A0917D01B0917E01B7FF1CC08EECC2D109
:1009E0008DE2C6D180917B0190917C01A0917D0127
:1009F000B0917E01B095A095909581959F4FAF4F96
:100A0000BF4F80937B0190937C01A0937D01B093B5
:100A10007E0104C08EECA6D18BE2AAD183ECA2D1D8
:100A20006091960170919701809198019091990140
:100A30002AE030E040E050E0ABD7DA01C901C6D08F
:100A40008AE396D189EC8ED16091A4017091A501C1
:100A50008091A6019091A7012AE030E040E050E0AB
:100A600097D7DA01C901B2D08AE382D18FEC7AD16B
:100A700060917B0170917C0180917D0190917E015C
:100A80002AE030E040E050E083D7DA01C9019ED08F
:100A90008091A8019091A901A091AA01B091AB0108
:100AA000B7FF1CC086ED5ED18DE262D18091A801B6
:100AB0009091A901A091AA01B091AB01B095A09528
:100AC000909581959F4FAF4FBF4F8093A801909312
:100AD000A901A093AA01B093AB0104C086ED42D155
:100AE0008BE246D180918A0190918B01A0918C017B
:100AF000B0918D01B7FF1CC08AED34D18DE238D1A1
:100B000080918A0190918B01A0918C01B0918D010F
:100B1000B095A095909581959F4FAF4FBF4F809313
:100B20008A0190938B01A0938C01B0938D0104C036
:100B30008AED18D18BE21CD18091920190919301A2
:100B4000A0919401B0919501B7FF1CC08EED0AD120
:100B50008DE20ED18091920190919301A091940128
:100B6000B0919501B095A095909581959F4FAF4F0D
:100B7000BF4F8093920190939301A0939401B093FF
:100B8000950104C08EEDEED08BE2F2D084EDEAD078
:100B90008CE3EED087EDE6D08091A801A6D08AE361
:100BA000E7D08BEDDFD080918A019FD08AE3E0D03F
:100BB0008FEDD8D08091920198D084EF91E0E8EC4D
:100BC000F0E03197F1F70197D1F785CCEF92FF92E2
:100BD0000F931F939C0168EE73E0C6D6182F092F60
:100BE000C90168EE73E0C0D6662311F480E302C049
:100BF000862F805DBDD0812F902F64E670E0B4D643
:100C0000F82EE92E812F902F64E670E0ADD6662392
:100C100011F480E302C0862F805DAAD08F2D9E2D17
:100C20006AE070E0A1D6362F8F2D9E2D6AE070E02D
:100C30009BD6182F332311F480E302C0832F805DED
:100C400097D0812F805D94D01F910F91FF90EF90EE
:100C500008950F931F939C0164E670E085D6182FCA
:100C6000092FC90164E670E07FD6662311F480E3A2
:100C700002C0862F805D7CD0812F902F6AE070E0CB
:100C800073D6362F812F902F6AE070E06DD6182F23
:100C9000332311F480E302C0832F805D69D0812F5C
:100CA000805D66D01F910F9108951F93282F64E6F1
:100CB0004FD6192F822F4CD6882311F480E301C020
:100CC000805D56D0812F6AE043D6282F812F40D6F1
:100CD000192F222311F480E302C0822F805D48D0B7
:100CE000812F805D45D01F9108951F93282F6AE0C2
:100CF0002FD6382F822F2CD6192F332311F480E3CF
:100D000002C0832F805D34D0812F805D31D01F9150
:100D10000895805D2DD008959AE69A95F1F7909800
:100D200092B3807F9F70982B92BB929A85E08A95B0
:100D3000F1F79298089592B3282F207F9F70292B66
:100D400022BB929A25E0922F9A95F1F7929892B34E
:100D50008295807F9F70982B92BB929A2A95F1F78B
:100D6000929808959AE69A95F1F79098E4DF08959D
:100D70009AE69A95F1F7909ADEDF08950F931F9304
:100D800081B3806F81BB889A899A8A9A80E991E0C1
:100D900028EC30E0F9013197F1F70197D9F780E3BA
:100DA000BBDF80E29EE40197F1F780E3B5DF00EA64
:100DB0001FE0C8010197F1F780E3AEDF88E2ACDF06
:100DC00088E2D0DF8CE0CEDF81E0CCDFC801019784
:100DD000F1F786E0C7DF1F910F910895CF93DF935E
:100DE000EC0102C02196C4DF88818823D9F7DF9106
:100DF000CF910895CF93DF93EC0104C0FE0184915D
:100E00002196B6DF88818823C9F7DF91CF910895B5
:100E10000F931F93CF93DF938C01862F90E0877001
:100E2000907023E0880F991F2A95E1F780649ADF7C
:100E3000C0E0D0E0F801EC0FFD1FE4918E2F98DFA9
:100E40002196C830D105B1F7DF91CF911F910F9155
:100E50000895A0E0B0E0EEE2F7E0D7C5DC012B0199
:100E6000FA019C91923008F439C1EB0188818230FB
:100E700008F433C1943069F4843009F02FC111961D
:100E80009C9111978981981709F428C1A0E6B0E0D8
:100E900025C1843009F421C18230A9F4923009F0CF
:100EA0001DC19A01AD0188E0EA010990AE01E90196
:100EB00009929E018150C1F7E201898111969C91AE
:100EC0008923818308C1923009F407C112962D90BD
:100ED0003C901397EB018A819B811496AD90BD9055
:100EE000CD90DC901797EC80FD800E811F819101E1
:100EF000281B390BB90137FF04C066277727621B0F
:100F0000730B603271050CF061C0121613066CF59C
:100F100037014801062E04C096948794779467940D
:100F20000A94D2F721E030E040E050E004C0220F04
:100F3000331F441F551F6A95D2F72150304040405F
:100F400050402E213F2140235123211531054105D9
:100F5000510521F021E030E040E050E079018A01C4
:100F6000E628F728082919293CC0232BD1F1260EA1
:100F7000371E35014601062E04C096948794779457
:100F800067940A94D2F721E030E040E050E004C0DA
:100F9000220F331F441F551F6A95D2F7215030404E
:100FA000404050402A213B214C215D212115310533
:100FB0004105510521F021E030E040E050E05901C9
:100FC0006A01A628B728C828D9280BC0821593051E
:100FD0002CF01C01AA24BB24650103C0EE24FF24CD
:100FE000870111969C91D20111968C91981709F462
:100FF00045C0992339F0A80197012A193B094C09EA
:101000005D0906C0A60195012E193F09400B510B41
:1010100057FD08C0118233822282248335834683A0
:1010200057831DC081E081833382228288279927DC
:10103000DC01821B930BA40BB50B84839583A683E1
:10104000B7830DC0220F331F441F551F24833583E0
:10105000468357838281938101979383828324817E
:10106000358146815781DA01C9010197A109B1098A
:101070008F5F9F4FAF4FBF4328F30BC091833382E5
:101080002282EA0CFB1C0C1D1D1DE482F5820683E6
:10109000178383E08083248135814681578157FF00
:1010A0001AC0C901AA2797FDA095BA2F8170907028
:1010B000A070B0705695479537952795822B932B46
:1010C000A42BB52B84839583A683B78382819381D8
:1010D000019693838283DF0101C0D201CD01CDB798
:1010E000DEB7E2E1AEC4A0E2B0E0E8E7F8E099C420
:1010F00069837A838B839C832D833E834F835887B8
:10110000E9E0EE2EF12CEC0EFD1ECE010196B701AA
:10111000A7D38E010F5E1F4FCE010596B801A0D355
:101120008A8991E089278A8BC701B801AE01475EA1
:101130005F4F8FDEC0D2A096E6E08FC4A0E2B0E0A1
:10114000E3EAF8E06EC469837A838B839C832D8302
:101150003E834F835887F9E0EF2EF12CEC0EFD1EF5
:10116000CE010196B7017CD38E010F5E1F4FCE01D9
:101170000596B80175D3C701B801AE01475E5F4F50
:1011800068DE99D2A096E6E068C4A0E2B0E0EAEC9E
:10119000F8E03BC469837A838B839C832D833E83F1
:1011A0004F835887CE010196BE01675F7F4F58D3AA
:1011B000CE010596BE016F5E7F4F52D39985923066
:1011C00088F089898230C8F0943019F4823051F463
:1011D00004C0843029F4923081F480E690E0C6C0E7
:1011E000923049F420E09A858A89981321E02A8771
:1011F000CE010996BBC0823049F420E09A858A89E5
:10120000981321E02A8BCE014196B0C02D843E84F4
:101210004F8458886D887E888F88988CEE24FF24B0
:101220008701AA24BB24650140E050E060E070E043
:10123000E0E0F0E0C10181709070892BE9F0E60CEC
:10124000F71C081D191D9A01AB012A0D3B1D4C1DF1
:101250005D1D80E090E0A0E0B0E0E614F704080532
:10126000190520F481E090E0A0E0B0E0BA01A90106
:10127000480F591F6A1F7B1FAA0CBB1CCC1CDD1C0E
:1012800097FE08C081E090E0A0E0B0E0A82AB92A6B
:10129000CA2ADB2A3196E032F10549F0660C771C48
:1012A000881C991C5694479437942794C3CFFA8589
:1012B000EA892B893C898B859C85280F391F2E5FF5
:1012C0003F4F17C0CA0181709070892B61F016954D
:1012D0000795F794E79480E090E0A0E0B0E8E82A72
:1012E000F92A0A2B1B2B76956795579547952F5F03
:1012F0003F4F77FDE7CF0CC0440F551F661F771F88
:1013000017FD4160EE0CFF1C001F111F21503040E3
:10131000403090E0590790E0690790E4790760F366
:101320002B8F3C8FDB01CA018F779070A070B0705B
:1013300080349105A105B10561F447FD0AC0E114AF
:10134000F1040105110529F0405C5F4F6F4F7F4F9D
:1013500040781A8EFE1711F081E08A8F4D8F5E8FD4
:101360006F8F78A383E0898FCE014996A4D1A09690
:10137000E2E167C3A8E1B0E0EFEBF9E04EC36983B7
:101380007A838B839C832D833E834F835887B9E078
:10139000EB2EF12CEC0EFD1ECE010196B70160D2B2
:1013A0008E010F5E1F4FCE010596B80159D22985D7
:1013B000223008F47EC03989323010F4B8017CC084
:1013C0008A859A8989278A87243011F0223031F45E
:1013D000231709F06EC060E670E06EC0343039F457
:1013E0001D861E861F86188A1C861B8604C0323006
:1013F00021F484E08987B7015FC02B853C858B8908
:101400009C89281B390B3C872B87ED84FE840F8534
:101410001889AD88BE88CF88D88CEA14FB040C05E7
:101420001D0540F4EE0CFF1C001F111F2150304021
:101430003C872B8720E030E040E050E080E090E007
:10144000A0E0B0E460E070E0EA14FB040C051D05C8
:1014500040F0282B392B4A2B5B2BEA18FB080C0990
:101460001D09B695A79597958795EE0CFF1C001F53
:10147000111F6F5F7F4F6F31710531F7DA01C901BD
:101480008F779070A070B07080349105A105B10580
:1014900061F427FD0AC0E114F1040105110529F0EA
:1014A000205C3F4F4F4F5F4F20782D873E874F87FF
:1014B000588BBE01675F7F4FCB01FDD06896EAE095
:1014C000C8C2A8E0B0E0E6E6FAE0A8C29B01AC0121
:1014D00083E08983DA01C9018827B7FD83959927BD
:1014E000AA27BB27B82E211531054105510519F44E
:1014F00082E0898339C08823A9F0203080E0380752
:1015000080E0480780E8580729F460E070E080E058
:101510009FEC2EC0EE24FF248701E21AF30A040B8D
:10152000150B02C079018A018EE1C82ED12CDC8214
:10153000CB82ED82FE820F831887C801B7016CD081
:1015400001971816190684F4082E04C0EE0CFF1C2F
:10155000001F111F0A94D2F7ED82FE820F831887B5
:10156000C81AD90ADC82CB82BA82CE010196A3D0F6
:101570002896E9E06FC2ACE0B0E0E0ECFAE055C2DA
:1015800069837A838B839C83CE010196BE016B5F56
:101590007F4F66D18D81823061F1823050F184308D
:1015A00021F48E81882351F12EC02F81388537FD9B
:1015B00020C06E812F3131051CF06623F9F023C065
:1015C0008EE190E0821B930B29853A854B855C85E3
:1015D00004C056954795379527958A95D2F7662387
:1015E000B1F050954095309521953F4F4F4F5F4F4B
:1015F0000EC020E030E040E050E009C02FEF3FEFA8
:101600004FEF5FE704C020E030E040E050E8B90170
:10161000CA012C96E2E025C2EF92FF920F931F932E
:101620007B018C0180E0E81680E0F80681E0080785
:1016300080E0180788F48FEFE816F1040105110522
:1016400031F028F088E090E0A0E0B0E017C080E042
:1016500090E0A0E0B0E012C080E0E81680E0F8067C
:1016600080E0080781E0180728F088E190E0A0E01A
:10167000B0E004C080E190E0A0E0B0E020E230E023
:1016800040E050E0281B390B4A0B5B0B04C0169559
:101690000795F794E7948A95D2F7F701E859FF4F39
:1016A0008081281B310941095109C9011F910F91FE
:1016B000FF90EF900895DF92EF92FF920F931F93A8
:1016C000FC01E480F58006811781D1808081823021
:1016D00048F480E090E0A0E1B0E0E82AF92A0A2B83
:1016E0001B2BA5C0843009F49FC0823021F4EE2466
:1016F000FF24870105C0E114F1040105110519F467
:10170000E0E0F0E096C0628173819FEF6238790774
:101710000CF05BC022E83FEF261B370B2A31310566
:101720002CF020E030E040E050E02AC0B801A701F2
:10173000022E04C076956795579547950A94D2F77F
:1017400081E090E0A0E0B0E004C0880F991FAA1FDC
:10175000BB1F2A95D2F70197A109B1098E219F21BC
:10176000A023B1230097A105B10521F081E090E00D
:10177000A0E0B0E09A01AB01282B392B4A2B5B2B60
:10178000DA01C9018F779070A070B0708034910534
:10179000A105B10539F427FF09C0205C3F4F4F4F29
:1017A0005F4F04C0215C3F4F4F4F5F4FE0E0F0E0E0
:1017B0002030A0E03A07A0E04A07A0E45A0710F062
:1017C000E1E0F0E079018A0127C06038710564F535
:1017D000FB01E158FF4FD801C7018F779070A070CF
:1017E000B07080349105A105B10539F4E7FE0DC054
:1017F00080E490E0A0E0B0E004C08FE390E0A0E0DF
:10180000B0E0E80EF91E0A1F1B1F17FF05C0169552
:101810000795F794E794319687E016950795F79426
:10182000E7948A95D1F705C0EE24FF248701EFEFF6
:10183000F0E06E2F679566276795902F9F77D79476
:10184000DD24D7948E2F8695492F462B582F5D295E
:10185000B701CA011F910F91FF90EF90DF9008959B
:10186000FC01DB01408151812281622F6F7770E0A2
:10187000221F2227221F9381892F880F822B282F36
:1018800030E0991F9927991F11969C931197211564
:101890003105A9F5411551056105710511F482E085
:1018A00037C082E89FEF13969C938E9312979A010C
:1018B000AB0167E0220F331F441F551F6A95D1F714
:1018C00083E08C930DC0220F331F441F551F1296C7
:1018D0008D919C911397019713969C938E931297D9
:1018E000203080E0380780E0480780E4580758F34C
:1018F00014962D933D934D935C93179708952F3F26
:10190000310579F4411551056105710519F484E03B
:101910008C93089564FF03C081E08C9312C01C92E5
:1019200010C02F57304013963C932E93129783E0AC
:101930008C9387E0440F551F661F771F8A95D1F758
:10194000706414964D935D936D937C9317970895EF
:10195000991B79E004C0991F961708F0961B881F01
:101960007A95C9F780950895AA1BBB1B51E107C062
:10197000AA1FBB1FA617B70710F0A61BB70B881F1F
:10198000991F5A95A9F780959095BC01CD010895AE
:1019900097FB092E05260ED057FD04D014D00AD08F
:1019A000001C38F450954095309521953F4F4F4F8E
:1019B0005F4F0895F6F790958095709561957F4FEC
:1019C0008F4F9F4F0895A1E21A2EAA1BBB1BFD014A
:1019D0000DC0AA1FBB1FEE1FFF1FA217B307E4070E
:1019E000F50720F0A21BB30BE40BF50B661F771F66
:1019F000881F991F1A9469F7609570958095909546
:101A00009B01AC01BD01CF0108952F923F924F92EF
:101A10005F926F927F928F929F92AF92BF92CF927E
:101A2000DF92EF92FF920F931F93CF93DF93CDB787
:101A3000DEB7CA1BDB0B0FB6F894DEBF0FBECDBFFF
:101A400009942A88398848885F846E847D848C84D0
:101A50009B84AA84B984C884DF80EE80FD800C81D9
:101A60001B81AA81B981CE0FD11D0FB6F894DEBFBC
:101A70000FBECDBFED010895DF93DD27B92FBF77EE
:101A800040E85FE31616170648075B0710F4D92FE6
:101A900051D09F938F937F936F93F6D0E6E2F0E05F
:101AA00013D037D02F913F914F915F9154D0DD23C8
:101AB00049F09058A2EA2AED3FE049EC5FE3D07884
:101AC0005D27F2D0DF9125C0DF93CF931F930F9353
:101AD000FF92EF92DF927B018C01689405C0DA2EB1
:101AE000EF0139D0FE01E894A591259135914591FA
:101AF0005591AEF3EF01D8D0FE019701A801DA9419
:101B000079F7DF90EF90FF900F911F91CF91DF91C8
:101B10000895092E0394000C11F4882352F0BB0F92
:101B200040F4BF2B11F460FF04C06F5F7F4F8F4FF5
:101B30009F4F08959B01AC0160E070E080E89FE357
:101B400019CC23D128F028D118F0952309F0FFC033
:101B500012C111244BC127D1A0F3959FD1F3950F4A
:101B600050E0551F629FF001729FBB27F00DB11D21
:101B7000639FAA27F00DB11DAA1F649F6627B00DB1
:101B8000A11D661F829F2227B00DA11D621F739F9A
:101B9000B00DA11D621F839FA00D611D221F749FA8
:101BA0003327A00D611D231F849F600D211D822FEF
:101BB000762F6A2F11249F5750408AF0E1F0882336
:101BC0004AF0EE0FFF1FBB1F661F771F881F915043
:101BD0005040A9F79E3F510570F0B9C007C15F3F63
:101BE000ECF3983EDCF3869577956795B795F79576
:101BF000E7959F5FC1F7FE2B880F911D96958795FE
:101C000097F9089511F40EF4B6C0A7C0D4D0D0F35C
:101C10009923D9F3CEF39F57550B87FFAFD00024FC
:101C2000A0E640EA900180585695979528F4805C8C
:101C3000660F771F881F20F026173707480730F4F4
:101C4000621B730B840B202931294A2BA69517940C
:101C50000794202531254A2758F7660F771F881FDC
:101C600020F026173707480730F4620B730B840BFC
:101C7000200D311D411DA09581F7B901842F915888
:101C8000880F9695879508959B01AC017ECA7DD0FB
:101C900030F082D020F031F49F3F11F41EF46BC07D
:101CA0000EF4E095E7FB53C0E92F7DD080F3BA171F
:101CB000620773078407950718F071F49EF595C0C5
:101CC0000EF4E0950B2EBA2FA02D0B01B901900157
:101CD0000C01CA01A0011124FF27591B99F0593F9B
:101CE00050F4503E68F11A16F040A22F232F342FE3
:101CF0004427585FF3CF469537952795A795F04031
:101D00005395C9F77EF41F16BA0B620B730B840B45
:101D1000BAF09150A1F0FF0FBB1F661F771F881FFD
:101D2000C2F70EC0BA0F621F731F841F48F4879555
:101D300077956795B795F7959E3F08F0B3CF939544
:101D4000880F08F09927EE0F97958795089597F9D2
:101D50009F6780E870E060E008959F3F31F0915008
:101D600020F4879577956795B795880F911D96957F
:101D7000879597F908959FEF80EC08959150504012
:101D8000660F771F881FD2F7089500240A9416164D
:101D9000170618060906089500240A941216130659
:101DA00014060506089557FD9058440F551F59F025
:101DB0005F3F71F04795880F97FB991F61F09F3F38
:101DC00079F087950895121613061406551FF2CF61
:101DD0004695F1DF08C0161617061806991FF1CFB1
:101DE00086957105610508940895E894BB276627D8
:0C1DF0007727CB0197F90895F894FFCFF6
:101DFC0000000000000000000001020203030303C6
:101E0C00040404040404040405050505050505057E
:101E1C00050505050505050506060606060606065E
:101E2C000606060606060606060606060606060646
:101E3C00060606060606060607070707070707072E
:101E4C000707070707070707070707070707070716
:101E5C000707070707070707070707070707070706
:101E6C0007070707070707070707070707070707F6
:101E7C0007070707070707070808080808080808DE
:101E8C0008080808080808080808080808080808C6
:101E9C0008080808080808080808080808080808B6
:101EAC0008080808080808080808080808080808A6
:101EBC000808080808080808080808080808080896
:101ECC000808080808080808080808080808080886
:101EDC000808080808080808080808080808080876
:101EEC000808080808080808080808080808080866
:081EFC0008080808080808089E
:00000001FF
